:020000040000FA
:0600000039EF18F01200B8
:0608000039EF18F01200B0
:060808007EEF0AF0120071
:060818002FEF0AF01200B0
:06082A0001009E300000F9
:08083000E801000008000000CF
:080838005AEC09F0FB0EDBCFC6
:10084000F3FFDB06F35000090AE0A8EC09F0FA0E0A
:1008500013EC0AF0F3E1151CF1E1010E01D0000EDA
:1008600089EF09F05AEC09F03B0EE12402E3E1685C
:10087000E652E16E010EDB6A020EDB6AF90EDBCF97
:10088000F6FFFA0EDBCFF7FFFB0EDBCFF8FF080019
:10089000F550DF6EDF5002E1ABEF08F0250EDF5CB4
:1008A00002E09EEF08F0030EDB6A040EDB6A050E21
:1008B000DB6A060EDB6A070EDB6AC2EC08F02D0E5F
:1008C000DF5C0CE02B0EDF5C09E0200EDF5C06E055
:1008D000230EDF5C03E0300EDF5C1AE1DF50300AEC
:1008E00014E0130A0FE0030A0AE00B0A05E0060A07
:1008F000E4E1030EDB80E1D7030EDB82DED7030EDB
:10090000DB84DBD7030EDB86D8D7030EDB88D5D795
:100910002A0EDF5C1BE1BEEC08F00CEC09F010E0E5
:10092000030EDB8006680768130EDBCF0BF0140E96
:10093000DBCF0CF0D6EC15F0040E04C0DBFF03D0C7
:10094000130EF5EC08F0C2EC08F00BD0090EDB6AD0
:1009500063EC09F003E0D7EC09F0FAD7090EF5ECE7
:1009600008F0030EDBB0DB982E0EDF5C1BE1C2EC5F
:1009700008F02A0EDF5C0BE1BEEC08F00CEC09F08D
:1009800003E1130E47EC09F0C2EC08F00BD0090E9E
:10099000DB6A63EC09F003E0D7EC09F0FAD7090E43
:1009A00047EC09F0680EDF5C07E1C2EC08F0680E66
:1009B000DF5C1DE1030E18D0740EDF5C17E07A0EC9
:1009C000DF5C14E0480EDF5C06E0540EDF5C03E001
:1009D0005A0EDF5C02E1020E07D06C0EDF5C03E012
:1009E0006A0EDF5C04E1010E9AEC09F0CBDBDF500C
:1009F0006E0A01E17FD31E0A01E192D1200A01E1D2
:100A00008FD13F0A01E149D11A0A01E146D10D0A0D
:100A100001E143D1200A01E140D13A0A01E13DD18F
:100A2000200A01E13AD1260A01E135D10D0A01E19E
:100A300032D11A0A01E1D9D0200A4AE0300A1FE077
:100A4000460A0EE0250A01E083D3D950F90FE96E7A
:100A5000FF0EDA20EA6E010EEE5E000EEE5AEE5A3E
:100A6000A8EC09F0250EE66E97DB03E1151C01E109
:100A700069D3A4EC09F001E26BD3DB2A69D3080E39
:100A8000DB6A040EDB50010806E2040EDB046CECAA
:100A900009F0DB508DDB080EDB5009E0030EDB5064
:100AA000010B05E174DB01E04DD3080EDB6A66DB68
:100AB000EFCFDFFF1CEC0AF003E1151C01E142D38C
:100AC000A4EC09F001E3DB2A62DB01E141D33AD374
:100AD000070EDB5002080FE1E8EC09F0030EAFEC63
:100AE00009F00E0EEECFDBFF0F0EEECFDBFF100E88
:100AF000EECFDBFF20D0F70EDBCF17F0F80EDBCF09
:100B000018F0020E175E000E185AF70E17C0DBFF22
:100B1000F80E18C0DBFF17C0E9FF18C0EAFF9FEC12
:100B200009F0166A0E0E14C0DBFF0F0E15C0DBFFB6
:100B3000100E16C0DBFF0E0EDBCFE6FF0F0EDBCF75
:100B4000E6FF100EDBCFE6FF99EC17F0E552E55219
:100B5000E552130E05C0DBFF140E06C0DBFF060EC8
:100B6000DB5005E0130EE3EC09F001E26CDB07EC6F
:100B70000AF002E2130E39DBCAEC09F006E0040EBB
:100B8000E3EC09F002E2050E30DB030EDBB005D02A
:100B9000FEDA01E0D7D2080EDB6A090EDB6A0E0E20
:100BA000DBCFF6FF0F0EDBCFF7FF100EDBCFF8FF2A
:100BB0000800F550DF6EDF5014E00DEC0AF011E292
:100BC0001CEC0AF003E1151C01E1BCD2BDDB01E322
:100BD000DB2A090EDB2AD9500E0FE96E000ECDDBA1
:100BE000E7D7D5DA01E1B4D2ADD2C8DA110EEECF33
:100BF000DBFF120EEDCFDBFF110EDBCFE6FF120E97
:100C0000DBCFE6FF8BEC17F0E552E552130EF3CF86
:100C1000DBFF140EF4CFDBFF060EDB5004E0130EF7
:100C2000D2DB01E210DB07EC0AF002E2130EDDDAA0
:100C3000B1DB05E0040EC7DB02E2050ED6DA030ED7
:100C4000DBB005D0A4DA01E07DD2080EDB6A090E24
:100C5000DB6A110EDBCFE9FF120EDBCFEAFFEFCF2D
:100C6000DFFFDF5014E0D9DB12E2E6DB03E1151C05
:100C700001E168D269DB01E3DB2A090EDB2A110EF0
:100C8000DB2ADBCFE9FF120EE8E3DB2AE6D77FDAC7
:100C900001E15ED257D2030EDB8E070EDB0410E1BA
:100CA00097DB040E5CDB0A0EEECFDBFF0B0EEECF04
:100CB000DBFF0C0EEECFDBFF0D0EEECFDBFF6CD0BB
:100CC000070EDB5003082CE1030EDBAE0DD0B4DAC7
:100CD000020E78DAEFCF14F0156A166A176A14AEAE
:100CE00039D01568166835D0F70EDBCF15F0F80E41
:100CF000DBCF16F0020E155E000E165AF70E15C069
:100D0000DBFFF80E16C0DBFF15C0E9FF16C0EAFFD7
:100D1000EFCF14F00A0E14C0DBFF0B0EDB6A38D0E5
:100D2000070EDB50020809E1030EDBAE04D05BDBEB
:100D300016AE10D00ED057DB0DD0030EDBAE12D0A6
:100D40007BDA020E3FDAFBDA166A176A15AE02D0BA
:100D500016681768E4DA0C0E16C0DBFF0D0E17C01C
:100D6000DBFF1AD0F70EDBCF16F0F80EDBCF17F053
:100D7000020E165E000E175AF70E16C0DBFFF80EB5
:100D800017C0DBFF16C0E9FF17C0EAFFD8DAC7DAE1
:100D90000C0EDB6A0D0EDB6A060EDB5005E1010E60
:100DA000F36E050EF3CFDBFF150EDB6A160EDB6A62
:100DB000D950370F146E000EDA20156E390E14C09C
:100DC000DBFF3A0E15C0DBFF380EDB6A080EDB6A6C
:100DD0000A0EB0DADF50780A12E0200A10E0280A82
:100DE0000CE0200A0AE03F0A06E00D0A02E0200AB1
:100DF00008E1020E05D0080E03D0080EDF26100E03
:100E000099DA030EDBBE02D0DB92DB94DB50800B61
:100E100024E08CDAD890030EEB50000A08E6000EAE
:100E2000EE5C000EEE58000EEE58000EEE5815E285
:100E300015DA09680A680B680C6853EC17F00A0E9B
:100E400000C0DBFF0B0E01C0DBFF0C0E02C0DBFF9E
:100E50000D0E03C0DBFF2D0E08D0030EDBA202D067
:100E60002B0E03D0DBA408D0200EF36E170EF3CFA9
:100E7000DBFF150EDB2A02D0170EDB6A050EDB50F6
:100E800003E1B9D901E189D08A0E146E300E156ED6
:100E9000000E166E070EDBCF17F0186A196A1A6A71
:100EA00017C009F018C00AF019C00BF01AC00CF0F6
:100EB000D5D9BEEC17F014500024F36E1550012064
:100EC000F46E16500220F86EF4CFF7FFF3CFF6FF62
:100ED0000800090EF5CFDBFF580EDF5C0FE1610E55
:100EE000F36E090E7DD90AE3200E146E090EDBCFD6
:100EF000E7FF1450E75E090EE7CFDBFF070EDBCFFD
:100F000014F0156A166A176A11DA14C009F015C0D0
:100F10000AF016C00BF017C00CF0EECF04F0EECFC5
:100F200005F0EECF06F0EFCF07F0BEEC17F007C0EC
:100F3000EDFF06C0EDFF05C0EDFF04C0EFFF390E69
:100F4000DBCFE9FFDB063A0EDBCFEAFF01E2DB068F
:100F5000090EDBCFEFFF150EDB2A4DD995E1030E0D
:100F6000DBA61DD06F0EDF5C06E1C3D918E3150EBA
:100F7000DB285DDA14D0780EDF5C09E0580EDF5C08
:100F800006E0620EDF5C03E0420EDF5C08E1020E69
:100F9000F36E160EF3CFDBFF02D0150EDB6A030EE5
:100FA000DB50100B0EE0040EDBCF14F0050EDB500F
:100FB000D880145406E2060EDB5003E1040EDB5029
:100FC00036DA97D90AE2050EDBCFE7FF150EDB50C4
:100FD000E75E050EE7CFDBFF02D0050EDB6A040EED
:100FE000DBCF14F0160E47D9D880145414E2160E35
:100FF000DBCFE6FF150EDBCFE6FF040EDBCFE6FF0F
:10100000050EDB50E552E75CE552D880E754E55227
:10101000D880E75461D9030EDB50010B0BE1080EB9
:10102000DB5008E0B4D801E08DD0080EDB50C0D80A
:10103000080EDB6A170EDB5007E08AD9170EF3D9CA
:1010400003E1151C01E17ED0160EDB5016E080D9BD
:10105000300EE66EA1D802E1151C74E079D9DFCF1D
:10106000E6FF11EC17F0E552E552E552F4CF15F02A
:101070000001F31C02E1151C65E0050EDBCF14F046
:10108000160EDB50D880145409E2050EDBCFE7FFC3
:10109000160EDB50E75E050EE7CFDBFF300EE66E87
:1010A000050ECDD94FE1390EDB2ADBCFE9FF3A0E31
:1010B00001E3DB2ADBCFEAFF090EEFCFDBFFDB50DA
:1010C0000EE046D9090EAFD902E1151C3BE0390EFE
:1010D000DB2ADBCFE9FF3A0EEDE3DB2AEBD757D86B
:1010E00031E1160EDBCFE6FF080EC5D8E552E72446
:1010F0005FD82ED0070EDB50030A1CE0010A14E073
:10110000030A07E07DD9DBCFEEFF020EDBCFEDFF58
:101110001FD0F7D8196A17AE02D0186819682ED8F0
:10112000BED819C0EEFF14D0ECD817BE186826D868
:10113000B6D80ED065D9DBCFEFFF0AD07DD905E157
:10114000151C03E1F368F46810D0FED801E3DB2A34
:101150007BD947EF04F0010EDBCF14F0020EDBCF9A
:1011600015F014C0F3FF15C0F4FFF56E3B0EE15C03
:1011700002E2E16AE552E16EF550CBD029D9020EC8
:10118000AFEF09F061D90800F550DF6E1200200EB4
:10119000E66E080E1FEF0AF011EC17F0E552E5526B
:1011A000E552F3CF14F0F4CF15F00001F31C120058
:1011B000146E156AD950010F4DD91450EE261550F2
:1011C000ED221200185E000E195AF70E18C0DBFF50
:1011D000F80E19C0DBFF18C0E9FF19C0EAFF1200C2
:1011E000DBCFF4FFF350F45C1200DB50E76E040E2B
:1011F000E7CFDBFF12000A0EDBCF14F00B0EDBCFC4
:1012000015F00C0EDBCF16F00D0EDBCF17F01450DF
:101210001510161017101200130EEECFDBFF140E70
:10122000EDCFDBFF130EDBCF14F0140EDBCF15F088
:101230000001800E15141200F70EDBCF18F0F80E27
:10124000DBCF19F01200050EDB50E66ED950130FFC
:1012500001D9E552E750EE6EED6A12000A0EDBCFBF
:1012600004F00B0EDBCF05F00C0EDBCF06F00D0EFD
:10127000DBCF07F01200DBCFE6FF150EDBCFE6FF7A
:10128000050EDB50E552E724E552E7241200DB505F
:10129000CED8010EF36E060EF3CFDBFF1200EE5038
:1012A000EFCFEAFFE96E16C0EEFF17C0EEFF18C0E1
:1012B000EEFF1200D9CFE6FFDACFE6FFE1CFD9FF8C
:1012C000E2CFDAFF1200DFCFE6FFE66AFCEC17F0B0
:1012D000E552E552F3501200E76E080EE7CFDBFF50
:1012E0001200EECF14F0EECF15F0EFCF16F0176A24
:1012F0001200050EDBCF14F0150EDB50D88014540D
:101300001200010EDBCF16F0020EDBCF17F0186AC9
:101310001200E552E5CFDAFFE7CFD9FF12000A0E3F
:1013200014C0DBFF0B0E15C0DBFF1200D9500A0FF3
:101330002AEF0AF0F36E070EF3CFDBFF1200EECFB9
:1013400014F0EFCF15F01200010EDB2A020E12008E
:10135000FC0EDBCFE6FFFD0EDBCFE6FF1200145ED6
:10136000000E155AF70E14C0DBFFF80E15C0DBFF98
:1013700014C0E9FF15C0EAFF1200DA20EA6EEF2A76
:10138000EECFF6FF000EEF22EECFF7FFEF22EECF0B
:10139000F8FF1200040EDBCFE6FF130EDB50E55220
:1013A000E75C9ADFDB5004DF060EDB501200090E0B
:1013B000DB500A0DF350DF24D00FE76E090EE7CFA4
:1013C000DBFFC2EF08F0DB50F36E050EF0EF08F024
:1013D000F70EDBCF14F0F80EDBCF15F01200DFCFE5
:1013E000E6FFCCEF08F028DF030EECDE71EF09F02A
:1013F0001CEC04F0E552E552E552E55200091200FA
:10140000BDDEEE50EFCFEAFFE96E010E1200130EC3
:10141000DB50F36E040EF0EF08F0040EDB50F36EB9
:10142000090EF0EF08F0DBCFE6FFCCEF08F0E76E37
:10143000050EE7CFDBFF12008BDFEFEF09F0DBCF0C
:10144000E6FF86DFF8EF09F0D950F90FE96EFF0EDD
:0E145000BDEF09F0E96E000EDA20EA6E120020
:02145E00D8CFE5
:10146000E4FFE0CFE4FFE46EDACFE4FFE2CFDAFF9F
:10147000E9CFE4FFEACFE4FFE6529E920101E82BB8
:10148000000EE9230101B8510101E85D0101B951E4
:101490000101E95926E3E86BE96B100E0101BA5D21
:1014A0001FE2B651EA6A860FE96E010EEA2280CF8A
:1014B000EFFFB651EA6A960FE96E010EEA2281CF7C
:1014C000EFFFB651EA6AA60FE96E010EEA2282CF5B
:1014D000EFFFB62B100EB65D01E1B66BBA2B01D053
:1014E000CA94E552E5CFEAFFE5CFE9FFE5CFDAFFA1
:1014F000E550E5CFE0FFE5CFD8FF1000DACFE4FFFD
:10150000E2CFDAFFE652E552E5CFDAFF1100896A51
:1015100092688A6A93688B6A9468FC0E8B1694169C
:1015200094848250040B01E0010E0101006F826B74
:10153000836BB76BB66BBA6BCA82CA80CA9CCA9AF5
:10154000CA88CA96FA0ECB6ED08E9D829F92F28E7A
:10155000F28C1200D9CFE6FFE1CFD9FF060EE126CB
:10156000010EDF6EDB6A020EDB6A030EDB6AD5EC6E
:101570000FF0060E0101F05D03E36D50020B01E078
:101580009AD00101BC5101E096D00101BA51000886
:1015900040E2B751EA6AA60FE96E010EEA22EF5067
:1015A000E66EE66AB751EA6A960FE96E010EEA2224
:1015B000EF50E66EE66AB751EA6A860FE96E010EF1
:1015C000EA22EF50E66EE66A280E146E300E156EB3
:1015D000166A14C0E6FF15C0E6FF16C0E6FF410E0E
:1015E000E66E010EE66E6AEC16F0F56E0B0EE15E2D
:1015F000F5500101B72B100EB75D01E1B76BBA07CB
:10160000410EE66E010EE66ED5EC10F0E552E552A5
:1016100052D0400EE66E010EE66E010EE66E95ECBF
:1016200010F0E552E552E552E76E010EE7CFDBFF21
:101630000101816BDBCF14F0000EE76E1418E8AEE9
:1016400002D0143403D0E750D880145405E2010EC0
:10165000DBCFE6FF3CD8E552D950040FE66E000E12
:10166000DA20E66EA2D8E552E552000924E0040E25
:10167000DBCFE6FF13D9E552000E0101E76E8119B9
:10168000E8AE02D0813503D0E750D880815513E20F
:101690000101BC5110E181C141F101010D0E426F08
:1016A0000A0E436F446B410EE66E010EE66ED5ECFA
:1016B00010F0E552E552F56E060EE15C02E2E16AD9
:1016C000E552E16EF550E552E7CFD9FF1200D9CFD0
:1016D000E6FFE1CFD9FFE652DF6AFE0EDB50DF5CAA
:1016E0005FE20101ED5123E10D0E146EDF50EA6A55
:1016F000010FE96E010EEA22EF50145C0BE00A0EB6
:10170000156EDF50EA6A010FE96E010EEA22EF5012
:10171000155C0DE1010EED6F01018251EA6A000FC7
:10172000E96E020EEA220D0EEF6E822B28D0DF50FA
:10173000EA6A010FE96E010EEA22EF500D081FE080
:10174000DF50EA6A010FE96E010EEA22EF500A0843
:1017500016E0DF50EA6A010FE96E010EEA22EF504F
:10176000E66E01018251EA6A000FE96E020EEA227A
:10177000E552E750EF6E0101ED6B0101822B010193
:101780008251146E156A800E141802E1000E1518AD
:1017900001E1826B8351825D01E102D0DF2A9DD796
:1017A000E552E552E7CFD9FF1200D9CFE6FFE1CFEE
:1017B000D9FF020EE126010E83C1DBFFDB500101E0
:1017C000825D0AE1FD0EDBCFE9FFFE0EDBCFEAFF13
:1017D000EF6A016B000E56D0DF6ADF50146E156A97
:1017E000D890155004E6800E145C000E155840E2A7
:1017F000010EDB50EA6A000FE96E020EEA22EF509A
:10180000E66EDF50EA6A010FE96E010EEA22E55248
:10181000E750EF6E010EDB2ADB50146E156A800E66
:10182000141802E1000E151802E1010EDB6A0D0E1C
:10183000146EDF50EA6A010FE96E010EEA22EF50E2
:10184000145C0FE1DF28E66EFD0EDBCFE9FFFE0E34
:10185000DBCFEAFFE552E750EF6E010EDBCF83F1FD
:1018600011D0010EDB50825D01E102D0DF2AB5D735
:10187000FD0EDBCFE9FFFE0EDBCFEAFFEF6A016B67
:10188000000E00D0F56E020EE15C02E2E16AE55264
:10189000E16EF550E552E7CFD9FF1200D9CFE6FF50
:1018A000E1CFD9FF2C0E0101025D07E0FE0EDB50F7
:1018B000020803E22C0E816F2FD0FE0EDB04EA6AD1
:1018C000010FE96E010EEA22EF500D0803E0210E30
:1018D000816F22D00151540A1DE0070A19E0120A53
:1018E00015E0170A11E01F0A0DE0060A09E00C0ACC
:1018F00005E0110A01E010D013D80ED067D80CD043
:10190000D1D80AD02CD908D054D906D05ED904D069
:1019100024DB02D007D800D0E552E7CFD9FF120070
:1019200087EF0AF0D9CFE6FFE1CFD9FF020EE1261B
:10193000010EDF6EDB6A030EE66ED9CFE6FFDACF6B
:10194000E6FF44D9E552E552E55205C084F106C0F0
:1019500085F1010EE66ED9CFE6FFDACFE6FF36D984
:10196000E552E552E552010E05C0DBFFDF50EA6AA1
:10197000010FE96E010EEA22EF500D0806E00101A9
:10198000815103E1230E816F15D00101815112E1D4
:101990008451851102E1CA940DD00A0E845D000EB7
:1019A000855903E20A0E846F856B84C1B8F185C145
:1019B000B9F1CA84F56E020EE15C02E2E16AE55219
:1019C000E16EF550E552E7CFD9FF1200D9CFE6FF1F
:1019D000E1CFD9FF050EE126010EF36E040EF3CF21
:1019E000DBFF010EE66ED950040FE66E000EDA2022
:1019F000E66EECD8E552E552E5520550DF6E010E79
:101A0000E66ED950040FE66E000EDA20E66EDED8E0
:101A1000E552E552E552010E05C0DBFFE66ED950F6
:101A2000040FE66E000EDA20E66ED0D8E552E552DD
:101A3000E552020E05C0DBFF010EE66ED950040F21
:101A4000E66E000EDA20E66EC1D8E552E552E552A8
:101A5000030E05C0DBFF040EDB50EA6A010FE96EDE
:101A6000010EEA22EF500D0806E00101815103E169
:101A7000230E816F0BD00101815108E1DF50926E7E
:101A8000010EDB50936E020EDB50946EF56E050E68
:101A9000E15C02E2E16AE552E16EF550E552E7CF22
:101AA000D9FF1200D9CFE6FFE1CFD9FF040EE1261E
:101AB000010EF36E030EF3CFDBFF010EE66ED9507D
:101AC000030FE66E000EDA20E66E80D8E552E5528E
:101AD000E5520550DF6E010EE66ED950030FE66E3B
:101AE000000EDA20E66E72D8E552E552E552010E9C
:101AF00005C0DBFFE66ED950030FE66E000EDA205C
:101B0000E66E64D8E552E552E552020E05C0DBFFF1
:101B1000030EDB50EA6A010FE96E010EEA22EF5074
:101B20000D0806E00101815103E1230E816F0BD006
:101B30000101815108E1DF50896E010EDB508A6E90
:101B4000020EDB508B6EF56E040EE15C02E2E16A80
:101B5000E552E16EF550E552E7CFD9FF12000101E1
:101B6000BC5126E18250E66EE66A8150E66EE66A76
:101B70008050E66EE66A280E146E300E156E166AF8
:101B800014C0E6FF15C0E6FF16C0E6FF410EE66E84
:101B9000010EE66E6AEC16F0F56E0B0EE15EF55086
:101BA000410EE66E010EE66ED5EC10F0E552E55200
:101BB00012000101BC5108E1580EE66E300EE66ECF
:101BC00013EC11F0E552E55212001200D9CFE6FFF6
:101BD000E1CFD9FF040EE126030EDB6A010181513A
:101BE00004E0056A066A076A2CD1FD0EDBCFE9FF27
:101BF000FE0EDBCFEAFFEF50EA6A010FE96E010E3D
:101C0000EA22EF502C0808E0815102E15E0E816F5C
:101C1000056A066A076A15D1FD0EDBCFE9FFFE0EE5
:101C2000DBCFEAFFEF2A2D0E146EFD0EDBCFE9FFAE
:101C3000FE0EDBCFEAFFEF50EA6A010FE96E010EFC
:101C4000EA22EF50145C0CE1010EF36E030EF3CFA9
:101C5000DBFFFD0EDBCFE9FFFE0EDBCFEAFFEF2A55
:101C6000050EE66ED9CFE6FFDACFE6FFFD0EDBCF3D
:101C7000E6FFFE0EDBCFE6FFF0D8F56E050EE15E67
:101C8000F550030EDB5021E0DFCF14F0010EDBCF67
:101C900015F0020EDBCF16F00A680B680C6814C052
:101CA00005F015C006F016C007F08DEC15F002C067
:101CB00014F003C015F004C016F014C0DFFF010ECD
:101CC00015C0DBFF020E16C0DBFFFC0EDB5026E169
:101CD000DFCF14F0010EDBCF15F0020EDBCF16F0D4
:101CE0001634000E161807E6D8807F0E1454000E26
:101CF0001554000E165401E28CD0D9CFE9FFDACF8B
:101D0000EAFF020ED880EB50FF0A06E6800EEE5C7A
:101D1000FF0EEE58FF0EEF5801E27BD0FC0EDB0405
:101D200024E1DFCF17F0010EDBCF18F0020EDBCF7E
:101D300019F01934000E191807E6D880FF0E175451
:101D4000000E1854000E195464E3D9CFE9FFDACF1E
:101D5000EAFF020ED890EB50000A06E6000EEE5C99
:101D6000000EEE58000EEF5854E3020E1A6EFC0EF1
:101D7000DB501A5C24E1DFCF1BF0010EDBCF1CF03F
:101D8000020EDBCF1DF01D34000E1D1807E6D880B3
:101D9000FF0E1B547F0E1C54000E1D543AE3D9CF86
:101DA000E9FFDACFEAFF020ED880EB50FF0A06E621
:101DB000000EEE5C800EEE58FF0EEF582AE3030E85
:101DC0001E6EFC0EDB501E5C2DE1DFCF1FF0010EFE
:101DD000DBCF20F0020EDBCF21F02134000E2118E2
:101DE00007E6D880FF0E1F54FF0E2054000E21542A
:101DF00010E3D9CFE9FFDACFEAFF020ED890EB501B
:101E0000000A06E6000EEE5C000EEE58000EEF58DB
:101E100009E20101815106E17E0E816F056A066AC1
:101E2000076A0FD0DFCF14F0010EDBCF15F0020EE2
:101E3000DBCF16F014C005F015C006F016C007F091
:101E400000D0F56E040EE15C02E2E16AE552E16E5B
:101E5000F550E552E7CFD9FF1200D9CFE6FFE1CF29
:101E6000D9FF020EE126FB0EDBCFE9FFFC0EDBCF34
:101E7000EAFFEE6AEE6AEE6A010EDB6AFA0EDB50EA
:101E8000F36E010EDBCFF4FFF350F45C58E2FD0E6D
:101E9000DBCFE9FFFE0EDBCFEAFFEF50EA6A010F6E
:101EA000E96E010EEA22EFCFDFFF300EDF5C45E383
:101EB000DF50390842E3FB0EDBCFE9FFFC0EDBCF3E
:101EC000EAFFEECF17F0EECF18F0EFCF19F00A0EC1
:101ED0000A6E0B6A0C6A17C005F018C006F019C02C
:101EE00007F08DEC15F002C017F003C018F004C025
:101EF00019F0300EDF5C1A6E1B6A1C6A17501A2428
:101F0000146E18501B20156E19501C20166EFB0EF7
:101F1000DBCFE9FFFC0EDBCFEAFF14C0EEFF15C0FC
:101F2000EEFF16C0EEFFFD0EDBCFE9FFFE0EDBCFAE
:101F3000EAFFEF2A010EDB2AA1D7000E02D0010E24
:101F400000D0F56E020EE15C02E2E16AE552E16E5C
:101F5000F550E552E7CFD9FF12000101815124E18C
:101F60000101BC5121E10101BA51E66EE66A1C0E85
:101F7000146E300E156E166A14C0E6FF15C0E6FF2B
:101F800016C0E6FF410EE66E010EE66E6AEC16F034
:101F9000F56E070EE15EF550410EE66E010EE66E3F
:101FA000D5EC10F0E552E55212000101EE51EF11AF
:101FB00004E1500EEE6FC30EEF6FEE07000EEF5B05
:101FC0000101F05108E0010E146E6D50020B01E0AA
:101FD000010E145C02E18B9015D0F00509E0020EB1
:101FE000F05D06E0030EF05D03E0050EF05D02E13A
:101FF0008B8008D0060EF05D05E10101EE51EF1176
:1020000001E18B70120082B403D0010E03D002D024
:06201000000E00D01200DA
:0A201600040120511F0B010801E036
:102020005BD02051600BE842E842E842E842E842D7
:10203000010801E051D0245103E0240501E04CD017
:102040002151230A48E0010A40E0030A30E0010A76
:1020500025E0240A22E0070A1FE0010A1CE0030A27
:1020600011E0010A01E038D00101030EE16F010126
:10207000CE0EE26F010EE36F0101F1930101080E34
:10208000E66F2AD00101030EE16F0101CE0EE46F6D
:10209000010EE56F21D020D01FD01ED00101030E0C
:1020A000E16F0101C30EE46F010EE56F15D0010170
:1020B000030EE16F0101C30EE26F010EE36F010138
:1020C000F1930101070EE66F07D00101030EE16FE6
:1020D00022C4CAF101D000D012000101C36BC20EAC
:1020E000C46F010EC56FC66BC76BC86B080EC96F96
:1020F000BC6BBB6B1A0E726E1E0E736E0401000E6B
:10210000166F050E176F400E146F0401196F080E3D
:102110001A6F050E1B6F880E186F0401480E1E6F94
:10212000050E1F6F400E1C6F1200D9CFE6FFE1CFE6
:10213000D9FF0101BB6B040118BF30D0FC0EDBCF0F
:1021400014F01951D880145403E2FC0E19C4DBFFBB
:102150000101BB6BFC0EDB50BB5D19E2BB51EA6AAF
:10216000080FE96E050EEA22EF50E66EBB51E76EEE
:10217000FD0EDBCFE9FFFE0EDBCFEAFFE750E926DD
:10218000000EEA22E552E750EF6EBB2BE3D70401C5
:10219000400E196F1817187D880E18130101BB51D6
:1021A00000D0E552E7CFD9FF1200D9CFE6FFE1CF4B
:1021B000D9FFE6520101BC5101E030D0DF6ADF2ACD
:1021C000DF50146E156A145002E1010E151801E17A
:1021D0000BD0FD0EDBCFE9FFDB2AFE0EDBCFEAFFE3
:1021E00001E3DB2AEF50EBE1DF50146E156AD950A2
:1021F000FD0FE96EFF0EDA20EA6E1450EE5E155008
:10220000ED5ADF06FD0EDBCFBDF1FE0EDBCFBEF1DA
:10221000DFCFC1F10101C26B010EBC6FE552E55287
:10222000E7CFD9FF1200D9CFE6FFE1CFD9FFE652C1
:102230000101BC5101E031D0DF6ADF2ADF50146EAA
:10224000156AFF0E141801E1155001E10CD0FD0EC6
:10225000DBCFF6FFDB2AFE0EDBCFF7FF01E3DB2A45
:102260000800F550EAE1DF50146E156AD950FD0FF1
:10227000E96EFF0EDA20EA6E1450EE5E1550ED5A4C
:10228000DF06FD0EDBCFBDF1FE0EDBCFBEF1DFCFF3
:10229000C1F10101010EC26FBC6FE552E552E7CFFB
:1022A000D9FF1200D9CFE6FFE1CFD9FFE6520401F2
:1022B0001CBF6BD0030E0101BC5D01E1BC6BBC51C6
:1022C00001E163D0020EBC5D06E104011D6B01015A
:1022D000030EBC6F54D0BC0552E1400E146E156A5B
:1022E000C151145C000E155803E2400EDF6E02D09F
:1022F000C1C1DFFFDFCF1DF4DF50C15DC16F480EEC
:10230000BF6F050EC06FC20515E1DF5012E0BDC101
:10231000F6FFBEC1F7FF0800F550BFC1E9FFC0C11D
:10232000EAFFEF6EBF2B000EC023BD2BBE23DF06DE
:10233000ECD713D0DF5011E0BDC1E9FFBEC1EAFF09
:10234000EF50BFC1E9FFC0C1EAFFEF6EBF2B000E27
:10235000C023BD2BBE23DF06EDD7C15110E1040120
:102360001D51146E156A400E141801E1155004E158
:102370000101020EBC6F03D00101030EBC6F400EC1
:1023800004011C171C7D880E1C13E552E552E7CF93
:04239000D9FF12005F
:0C23940004012051600BE842E842E842DE
:1023A000E842E842000901E055D02151070A51E016
:1023B0000B0A4FE0070A40E0010A2CE00B0A28E074
:1023C000020A26E0030A22E0080A12E0010A0EE0EF
:1023D0000F0A0AE0030A01E03CD00101010EE16F9F
:1023E0000101040EF06F36D036D834D090D832D0F8
:1023F0000101010EE16F0101F20EE26F010EE36FC8
:102400000101F1930101010EE66F24D0A8D822D07A
:10241000F4D820D00101010EE16F04012451010123
:10242000E26FE36BF30EE227010EE3230101F19368
:102430000101010EE66F0ED00101010EE16F0401F2
:102440002451EA6AF30FE96E010EEA2222C4EFFF7B
:1024500001D000D01200800E0401205D57E123510D
:10246000030A34E0010A10E0030A01E04DD0010143
:10247000010EE16F0101060EE26F2C0EE36F120EEA
:102480000101E66FE76B40D00101010EE16F04012D
:102490002251F66EF76AD890F636F736C70EF62652
:1024A0002C0EF7220900F5CFE2F10A00F5CFE3F197
:1024B000020E0101F76AE225F66EE351F7220900E8
:1024C000F5CFE6F10A00F5CFE7F11ED00101010ECC
:1024D000E16F04012251F66EF76AD890F636F736AE
:1024E000CB0EF6262C0EF7220900F5CFE2F10A00FA
:1024F000F5CFE3F1E2C1F6FFE3C1F7FF0800F550C5
:102500000101E66FE76B00D00101F18312000101C8
:10251000010EE16F0F0EE66E710EE66E0F0EE66EA7
:1025200078EC15F0E552E552E552010EE66EF30E39
:10253000E66E010EE66E78EC15F0E552E552E552D6
:1025400022C4F2F10401225104E10101050EF06FF1
:1025500005D00101060EF06F6DEC10F012000401C1
:10256000286B296B040120511F0B020A14E0030A97
:102570000EE0010A01E033D00101010EE16F040118
:1025800028810101F1A102D00401288328D0010192
:10259000010EE16F24D00101010EE16F040124510D
:1025A0000F0B080DF350156A000F146E040E152260
:1025B0002451800B01E0010E040DF350010114249D
:1025C000E46F000E1520E56FE4C1E9FFE5C1EAFF05
:1025D000EF50040B03E00401010E286F00D001014D
:1025E000E1050AE10101280EE26F040EE36F01012B
:1025F000F1930101020EE66F12000401220510E1C1
:1026000020511F0B00090CE10101010EE16F030EC7
:102610000401215D03E10101F18102D00101F19189
:10262000040122513AE120511F0B020836E12451E6
:102630000F0B000932E00101010EE16F040124518A
:102640000F0B080DF350156A000F146E040E1522BF
:102650002451800B01E0010E040DF35001011424FC
:10266000E46F000E1520E56F030E0401215D07E104
:10267000840EE4C1E9FFE5C1EAFFEF6E0ED024AF9E
:1026800006D0E4C1E9FFE5C1EAFFEF6A06D0880E93
:0C269000E4C1E9FFE5C1EAFFEF6E1200B3
:04269C006C5002E09C
:1026A000000E01D0010E00090BE0040100513C0BAB
:1026B000E842E8420D0802E10CD801D040D808D029
:1026C0006C5002E0000E01D0010E040901E047D871
:1026D0001200D9CFE6FFE1CFD9FFE6520101E06B4E
:1026E000E16BE66BE76BCAEC11F0DF6ADF50146E4A
:1026F000156A010E145C000E15581BE20101E15130
:1027000001E017D0F76ADF34FE0BF736F66ED10E14
:10271000F6262C0EF7220900F5CF14F00800F5CFAD
:1027200015F004D015C0FAFF1450F96EFBDFDF2A54
:10273000DDD7E1D8E552E552E7CFD9FF1200020E0E
:102740000101E05D0AE198D8040100BD03D0C80E84
:10275000006F02D0880E006F01D013D91200040E52
:102760000101F05D0AE122C46EFF6E50000803E231
:10277000050EF06F02D0030EF06F0101E0050AE1D3
:102780000BD8040104BD03D0C80E046F02D0880E1C
:10279000046F01D0F6D81200D9CFE6FFE1CFD9FF00
:1027A000020EE1260101080EE65D000EE75905E282
:1027B000E6C1DEFFE7C1DDFF03D0080EDE6EDD6A95
:1027C000040104930491010EDB500413DFCF05F4E0
:1027D000000EDB500101E65F010EDB50E75B280EC7
:1027E000E46F040EE56F0101F1A31ED0D9CFE9FF1C
:1027F000DACFEAFFEE50ED1016E0E2C1F6FFE3C1DA
:10280000F7FF0800F550E4C1E9FFE5C1EAFFEF6E0C
:102810000101E42B000EE523E22BE323DF06010E8A
:1028200001E2DB06E3D71CD0D9CFE9FFDACFEAFF1C
:10283000EE50ED1015E0E2C1E9FFE3C1EAFFEF5011
:10284000E4C1E9FFE5C1EAFFEF6E0101E42B000EF0
:10285000E523E22BE323DF06010E01E2DB06E4D7EA
:10286000F56E020EE15C02E2E16AE552E16EF550BE
:10287000E552E7CFD9FF1200D9CFE6FFE1CFD9FF6C
:10288000020EE126030E04010015E76E010EE7CFEC
:10289000DBFF01C4DFFFDE500101E627DD50E72347
:1028A000280EE26F040EE36FD9CFE9FFDACFEAFF1B
:1028B000EE50ED1014E0E2C1E9FFE3C1EAFFEF5092
:1028C000E4C1E9FFE5C1EAFFEF6EE42B000EE5236A
:1028D000E22BE323DF06010E01E2DB06E5D7F56E0E
:1028E000020EE15C02E2E16AE552E16EF550E5526A
:1028F000E7CFD9FF12000101E1510CE10401080EFC
:10290000016F200E026F040E036F840E006F04012E
:10291000046F35D0040120AF22D00101E65104013B
:10292000265D0101E7510401275904E226C4E6F1BE
:1029300027C4E7F131DF0101010EE06F0401080E49
:10294000016F200E026F040E036F800E006F0401F2
:10295000280E066F040E076FC80E046F10D0010119
:10296000020EE06F0401056BC80E046F0401080E2F
:10297000016F280E026F040E036FC80E006F6D9872
:1029800012000101E06B0401080E016F200E026FBE
:0E299000040E036F880E006F0401046B12002A
:02299E006DA624
:1029A0000FD802D06DB613D80101F00508E16DBA59
:1029B00006D0686A696A69806988020EF06F120041
:1029C0006D6A696A6D860101010EF06F12006D6A11
:1029D000696A0101F06B1200E7EF14F00101F05198
:1029E00001E13AD06850040B04E06950040B01E0A7
:1029F0003CD86DB231D06850010B04E06950010B36
:102A000001E054D86850100B04E06950100B01E04D
:102A100024D86850400B04E06950400B01E03BD8DB
:102A20006850200B04E06950200B01E036D8685054
:102A3000020B04E06950020B01E036D8030E0101DD
:102A4000F05D01E209D06850080B06E06950080B00
:102A500003E04EEC13F068961200698468986D826A
:102A6000A19AA08A0300A09A12006D9269946894BA
:102A700012000101F1A10ED0F8DF6D840101080EF2
:102A8000F46F070EF56FF407000EF55BF451F511C6
:102A9000FAE16D941200689C120070A003D0C1ECA2
:102AA00014F07090689A1200689212006A6A686A5C
:102AB0009F0E6B6E7B0E696E6E6A0F0EE66E710E68
:102AC000E66E0F0EE66E14D8E552E552E552160E8C
:102AD000706E68A602D06896FCD76D98C1EC14F0B1
:102AE0000101F1910101F26B0101030EF06F12007F
:102AF000D9CFE6FFE1CFD9FFFD0EDBCFE9FFFE0E18
:102B0000DBCFEAFFFC0EDB5004E0EE6AFC0EDB06D6
:0A2B1000F9D7E552E7CFD9FF120014
:062B1A0007C013F006C025
:102B200012F005C011F005500A02F4CF03F0F3CF04
:102B300002F006500B02F4CF05F0F3CF04F00A02C6
:102B4000F3500326F4500422E86A052211500B02C8
:102B5000F3500326F4500422E86A052207500A02C3
:102B6000F3500426F450052207500B02066AE86A67
:102B70000622F3500526F450062211500C02F350A1
:102B80000426F4500522076AE86A0622072212503A
:102B90000C02F3500526F4500622E86A072213506F
:102BA0000C02F3500626F4500722000C07C013F065
:102BB00006C012F006500B02F4CF05F0F3CF04F07C
:102BC00007500C02F4CF07F0F3CF06F00B02F350DE
:102BD0000526F4500622E86A072212500C02F35030
:102BE0000526F4500622E86A07220CAEFCEF15F029
:102BF0001250065E1350075A13AE000C0B50065EBF
:062C00000C50075A000C05
:0A2C06001201000202000008D804C9
:102C10000A000000010200010902430002010080D5
:102C20003209040000010202010005240010010421
:102C30002402020524060001052401000107058283
:102C40000308000209040100020A0000000705034E
:102C50000240000007058302400000040309043419
:102C6000034D006900630072006F00630068006933
:102C7000007000200054006500630068006E006F63
:102C8000006C006F0067007900200049006E00634F
:102C9000002E003403430044004300200052005340
:102CA000002D00320033003200200045006D007519
:102CB000006C006100740069006F006E0020004429
:102CC0000065006D006F00182C182C5B2C5F2C9396
:032CD0002C16209F
:0C2CD400D9CFE6FFDACFE6FFE1CFD9FF51
:102CE000E2CFDAFFE652E652E652E652D950F90F49
:102CF000146EFF0EDA20156E020E14C0DBFF030EF9
:102D000015C0DBFF020EDBCFE6FF030EDBCFE6FFD5
:102D1000F90EDBCFE6FFFA0EDBCFE6FFFB0EDBCFD3
:102D2000E6FFD950FC0FE66EFF0EDA20E66E32ECBD
:102D300004F0F56E070EE15C02E2E16AE552E16E35
:102D4000F550F3CFDEFFF4CFDDFFFC0EDBCFE9FF64
:102D5000FD0EDBCFEAFFEF6ADECF14F0DDCF15F01A
:102D600014C0F3FF15C0F4FFF56E040EE15C02E23F
:102D7000E16AE552E16EF550E552E5CFDAFFE7CFC3
:042D8000D9FF120065
:0C2D84002A0EF66E080EF76E000EF86EB8
:102D900001010900F550DB6F0900F550DC6F03E11C
:102DA000DB6701D03DD00900F550D66F0900F55022
:102DB000D76F0900F550D86F09000900F550E96E8A
:102DC0000900F550EA6E090009000900F550D96FB5
:102DD0000900F550DA6F09000900F6CFDDF1F7CFF1
:102DE000DEF1F8CFDFF1D6C1F6FFD7C1F7FFD8C1CA
:102DF000F8FF0101D95302E1DA5307E00900F55069
:102E0000EE6ED907F8E2DA07F9D7DDC1F6FFDEC1C9
:102E1000F7FFDFC1F8FF0101DB07000EDC5BBFD766
:022E200012009E
:0E2E2200D9CFE6FFDACFE6FFE1CFD9FFE2CF4E
:102E3000DAFFFB0EDBCF14F0FC0EDBCF15F0000148
:102E4000800E15141AE1FB0EDBCFE9FFFC0EDBCF81
:102E5000EAFFEECFF3FFEDCFF4FFEE2A000EEF22F4
:102E6000F3CFE9FFF4CFEAFFFD0EDBCFEFFFEF502A
:102E7000156AF36E15C0F4FF10D0FB0EDB50FE0890
:102E800006E1FD0EDBCFE6FF1EEC18F005D0FD0ECF
:102E9000DBCFE6FF4EEC18F0E552E552E5CFDAFF66
:062EA000E7CFD9FF12008C
:0A2EA60004500902F3CF00F0F4CF4E
:102EB00001F00A02F3500126000EF420026E0450C5
:102EC0000B02F3500226000EF420036E04500C0295
:102ED000F350032605500902F3500126F450022254
:102EE000000E032205500A02F3500226F45003227A
:102EF00005500B02F350032606500902F350022638
:102F0000F450032206500A02F35003260750090228
:062F1000F350032612003D
:0A2F1600FE0EE3CFE9FFFF0EE3CF4C
:102F2000EAFFF36AF46AEE5203E0F34AF42AFBD7AD
:102F30001200FF0EE3CFF8FFE552FF0EE3CFF7FFDD
:102F4000E552FF0EE3CFF6FFE552E66AE66AE66A6F
:102F50000900F55209E0FD0EE32A05E1FE0EE32A21
:102F600002E1FF0EE32AF4D7FD0EE3CF05F0FE0EDB
:0C2F7000E3CF06F0FF0EE3CF07F01200E5
:042F7C00036A026A78
:102F8000016A006A200EE76ED890043605360636D0
:102F9000073600360136023603360950005C0A5007
:102FA00001580B5002580C50035809E30950005EB9
:102FB0000A50015A0B50025A0C50035A042AE72EA9
:042FC000E4D7120040
:0C2FC40005D810D8AAEC0AF0FCD71200C7
:102FD0000F0EC112140E6F6E0101F06B0101F16B47
:102FE0000101F26B87EF0AF0CFEC14F06FBE02D054
:082FF000EEEC14F052EF11F0B9
:082FF800F36AF46AFF0EE12404
:10300000E96EFF0EE220EA6EED6607D02F0EEF6448
:0C30100004D03A0EEF6001D0F32A120049
:04301C005374617414
:1030200075733D25690A0D00492C253033692C251F
:0B3030003033692C253033690A0D0095
:04303C00FF0EE35050
:10304000ACBA04D0AF6AAB8EAC8A949CACA2FED76B
:08305000AD6EF36EF46A12008C
:08305800554257204657204461
:103060002056657273696F6E20312E312E300A0D35
:01307000005F
:0E30720013EE00F023EE00F0F86A0F9CC2ECA3
:0A30800016F0E2EC17F0FDD7120085
:06308A0030313233343511
:0B309000363738396162636465660002
:02309C00120020
:02309E00000030
:0630A000410000000000E9
:00000001FF
